:10000000830100308A0004288301B72B9100921BE2
:10001000102812088A001108910A0319920A820016
:100020008313121883171108910A8400000808002E
:10003000423479342034503461346F346C346F344A
:1000400000344C3427346934723472346934673480
:10005000613474346F3472346534203430342E3467
:040060003134003403
:1006AA008C00831205110C08803E822B83120511DF
:1006BA00013082230230612B8D0004308E005330CA
:1006CA008F008F0B662B8E0B642B8D0B622B831284
:1006DA000800831205157A2B0D0892000C088C0A63
:1006EA0003198D0A0620831282230D0892000C0832
:1006FA000620003803190800712B8E000E0E0F39E0
:10070A00831290000608F0391004860085158511B9
:10071A000E080F3990000608F03910048600851576
:10072A0085110D308F008F0B982B831208008C00D7
:10073A00831205150C0E0F3990000608F0391004C3
:10074A008600851585110C080F3990000608F039C6
:10075A0010048600851585110D308D008D0BB32B85
:10076A008312080083168101810A03308500D03084
:10077A0086008312DA230030552321308C000030A2
:10078A008D006E234030552318308C0000308D00C8
:10079A006E2386128518D62B8612FA3083126123AD
:1007AA00CF2B051ACF2B8616D22B831205110F30A9
:1007BA00612303308600851585110530612385156F
:1007CA00851121308C008C0BE82B8312851585113D
:1007DA000530612302308600851585110D308C00A5
:1007EA008C0BF52B283083128223083082230F309A
:0607FA0082230630822B71
:02400E0011009F
:00000001FF
